:10000000B6C018951895189518951895189583C524
:10001000189518951895189518959F93AF939295E4
:10002000A92FAF7EA06EA5BBAD989295A92FAF7EEC
:10003000A06EA5BBAD98AF919F911DD008959F93E1
:10004000AF939295A92FA06FA5BBAD989295A92FBC
:10005000A06FA5BBAD98AF919F910DD008959F93D0
:1000600098E2DBDF9CE0D9DF98E2D7DF91E0D5DFD3
:1000700008D09F9108952F9322E32A95F1F72F91AD
:1000800008951F932F9319E02FEF2A95F1F71A95F2
:10009000D9F72F911F91089591E0BFDFF2DF089506
:1000A0000609090600000000100808040A0A1100E9
:1000B00090E4B3DFF0E0E0EA50E1C895902DBFDFB7
:1000C00091915A95D1F790E8A8DF0895AF93BF9327
:1000D000A92F90E8A2DFB0E2B03111F498EA9DDFD9
:1000E00099279FBBAEBBE09A9DB3A9DFA395BA95B4
:1000F00099F7BF91AF9108955F930F9290E88DDFCC
:1001000050E2503111F498EA88DFC895902D97DFBE
:1001100031965A95B1F70F905F910895AA20F1F3A7
:100120009A2DAA2408959A2DAA240895F894222499
:1001300012BE78945F9904C02314E1F7689402C05A
:100140009CB1E89408950F9307E109B908E10AB951
:100150000F9108950F9300270AB90F9108955D9BA1
:10016000FECF9CB908955F9BFECF9CB10895AA2451
:10017000BB24FF240FE50DBF02E00EBF06E001BB6C
:1001800008E702BB0FE304BB04E003BF08EB102E3B
:1001900012BE02E009BF08EC302E61DF89DF7894DF
:1001A000F8E1E0E4A9DF98ECAFD4AED4ADD4FF24FD
:1001B00021E00DD5B3DF983079F0923021F4223070
:1001C000C1F32395F6CF943021F4213091F32A9591
:1001D000F0CF913071F7EDCFF8E1E0EA8DDF50E03C
:1001E0009CE01BDF9AEC19DF952F9F5C28DF9BDFDB
:1001F0009130E9F298EC88D496DF9130C1F250FD4D
:1002000083D491DF913099F251FD7ED48CDF91300F
:1002100071F251FD79D487DF913049F29BDFB1D380
:1002200082DF913021F28FDFD8D356F453955430CA
:10023000B9F6F8E1E0EC60DF98EC66D465D4B7CFAE
:1002400011D4F8E1E0E058DF53E0992469E0E2D30B
:100250003EF108D42EF15A95C1F792E0DEDE11DFAF
:100260002227BED4992469E0D5D3D6F0FBD3C6F0BB
:100270005ADF9923B1F3923021F4243091F323957E
:10028000F0CF943021F4203061F32A95EACF9830F2
:1002900041F7BED4243029F78ACF11D091D0FDCFB9
:1002A00086CF5F9350E1112319F098E110E002C06E
:1002B0009CE111E0B2DE5A95E9F75F9108951127AC
:1002C000EBDE992467E0A6D35EF3CCD34EF3E3E6EE
:1002D000FF273327343099F06C3F89F40E2F0056F6
:1002E000071520F422D0ED5F3395F4CF992469E00F
:1002F00091D3B6F2B7D3A6F2FF27E3E6EBCF99246A
:1003000069E088D36EF2AED35EF20DDF9923B9F3C4
:100310009830A9F3913011F0C4DFF1CFBDDE08951C
:10032000992466E077D3C6F108950F939F935F9366
:10033000FF93EF939CE830FD9CEC31FD985E6DDE01
:1003400094E06BDE0281EF93FF9390E306FD91E36F
:1003500076DE90E307FD91E372DE9DE270DE0F73BF
:10036000E02EDD24C0D3905D6ADEBDD3905D67DEF4
:100370009DE265DEFF91EF91D080E18055E0B3D33F
:10038000905D5DDE5A95D9F796E047DEEF91FF91DB
:100390005F919F910F9108950ACF992465E03AD318
:1003A000DEF360D3CEF3F8E1E0E2A6DE992469E063
:1003B00031D396F357D386F3B6DE9923B9F3089574
:1003C000CC24C39469DE9C2C69E224D32EF34AD357
:1003D0001EF3623051F4F0E0E0E6B0E0A0EE50E849
:1003E00001910D935A95E1F731C0643FD1F4F0E0EB
:1003F000E3E6B0E0A3EE50DE94E00FDE552797E889
:1004000051FD97EC50FD985F08DE9D914D90519005
:1004100088D000279D91A90FB01F5395543079F7CC
:1004200015C0673E99F4F0E0E3E636DE94E0F5DDD2
:10043000552797E851FD97EC50FD985FEEDD9191BF
:10044000419051906ED05395543099F76CDE9030B6
:1004500009F4B9CF923059F4C3941EDE992469E0AF
:10046000D9D2BEF091E050D3FDD29EF0ACCF943003
:1004700059F4CA9411DE992469E0CCD256F091E087
:1004800043D3F0D236F09FCF913009F09CCF04DEF9
:1004900008958DCE01DE9CE0C0DD6627112755272B
:1004A0009924B8D2B6F3DED2A6F390E850FD90ECD2
:1004B00051FD985EB2DDE0E6F0E00191043050F0CD
:1004C0000350702E01910191772021F07A9491913F
:1004D000B6DDFACF69E05395543011F7992469E0FD
:1004E00099D2BEF2BFD2AEF21EDE9923B9F391309B
:1004F00021F0983099F3D5DEF1CF08959A3010F4B9
:10050000905D02C09A509F5B08959F939F70F6DFA5
:1005100096DD9F919695969596959695EFDF8FDD52
:100520000895983811F417D20895993811F407D224
:100530000895943811F4EDD10895903911F4DAD179
:100540000895933211F4D6D10895913811F49DD1C4
:1005500008959B3811F4FAD008959B3011F45CD1C2
:100560000895923911F458D108959F3811F473D138
:1005700008959C3811F418D108959D3811F4C1D014
:100580000895913111F4B4D00895913011F49FD0B1
:100590000895953011F47ED00895963011F46FD0FF
:1005A0000895903111F4D7D10895923011F456D0B6
:1005B0000895983111F445D008959F3011F4BFD1BA
:1005C0000895933011F42DD00895943011F40FD084
:1005D0000895953811F474D108959F9390E22FDD1A
:1005E000952D93DF942D91DF9F918FDF089590E0FB
:1005F00026DD90E224DDD42CE52C0E2D0F3730F4CF
:100600000FE70E19E02E0DE20F9304C00F57E02EF6
:1006100000E20F9398D267D201E0A4D29F910FDD40
:10062000089590E00CDD9CE30ADD90E208DDD42C17
:10063000E52C89D2EE0CDD1C56D255D201E092D2C7
:10064000089590E2FCDC91E4FADC90E2F8DCD42C32
:10065000E52C79D248D202E085D2089590E2EFDC11
:1006600095E2EDDC90E2EBDCD42CE52C6CD2EE0CC8
:10067000DD1C39D238D237D20FEF74D2089596E507
:10068000DEDC90E2DCDCD42CE52C5DD22CD202E066
:1006900069D2089590E2D3DC90E2D1DC93E4CFDC20
:1006A00090E0CDDCD42CE52C0E2D043630F404E69D
:1006B0000E19E02E0DE20F9304C00456E02E00E266
:1006C0000F9341D201E04ED29F91B9DC08959DE491
:1006D000B6DC90E5B4DC92E5B2DC90E2B0DCD42C80
:1006E000E52C31D2EE0CDD1CFED10FEF3BD208958C
:1006F00090E2A5DCA4DCA3DC952DA1DC942D9FDC8D
:100700000895BF93AF935F9358E090E298DC5A95B9
:10071000E1F796E082DC5D91552049F00D910030C3
:1007200011F0033009F45A945A95B1F709C058E012
:100730009D91903029F0933019F081DC5A95C1F7E2
:1007400094E06BDC5F91AF91BF910895BF93AF933D
:10075000DF93CF939DE473DC90E571DC92E56FDC71
:1007600090E26DDC9D919A9501E0D02E00E0E02EA4
:10077000A6D1EF929E2DE52CDD24A1D10027AE0D50
:10078000B01FCD91DD91DC2EDD1AE92EDCD19F91D9
:1007900096D1CE19EC2ED42CD6D10FEFE3D1CF9138
:1007A000DF91AF91BF910895BF93AF93DF93CF9344
:1007B00090E245DC90E243DC93E441DC90E03FDCF6
:1007C0009D919A9501E0D02E00E0E02E78D1EF9235
:1007D0009E2DE52CDD2473D10027AE0DB01FCD91E9
:1007E000DD91DC2EDD1AE92EAED19F9168D1CE19B4
:1007F000C41528F44C1AE42C0DE20F9304C0C4195C
:10080000EC2E00E20F930FEFADD19F9118DCCF914A
:10081000DF91AF91BF91089591E011DC90E20FDC80
:10082000D42CE52C0E2D003830F400E80E19E02E03
:100830000DE20F9304C00058E02E00E20F9383D125
:1008400000E1E00E07E2D01E4ED14DD102E08AD188
:100850009F91F5DB089590E0F2DB90E2F0DBD42C81
:10086000E52C0E2D003830F400E80E19E02E0DE2D4
:100870000F9304C00058E02E00E20F9364D133D1EF
:1008800001E070D19F91DBDB089590E2D8DB95E227
:10089000D6DB90E2D4DBD42CE52C55D124D123D166
:1008A000DF92EF9220D14D2C5E2CEF90DF90EE0C7A
:1008B000DD1CEE0CDD1CE518D40801E053D10895D1
:1008C00090E2BDDB96E5BBDB90E2B9DBD42CE52CF6
:1008D0003AD1DF92EF9207D14D2C5E2CEF90DF9052
:1008E000EE0CDD1CEE0CDD1CE518D408FCD002E09B
:1008F00039D1089598E6A3DB9FE2A1DB9CE69FDB5C
:1009000090E29DDBD42CE52C1ED1EDD001E02AD164
:10091000089590E094DB9CE392DB90E290DBD42C92
:10092000E52C11D1DF92EF92EE0CDD1CEE0CDD1CFC
:100930000F91E00E0F91D01E01E014D1089593E7BE
:100940007EDB9DE67CDB90E27ADBD42CE52CFBD0D1
:1009500002E008D108950F935F9301E058E0942DD1
:10096000902311F490E206C0952D902311F490E3AA
:1009700001C091E364DB000F5A9589F75F910F91F5
:1009800008950F934F935F932F93899A8A9A4427E0
:100990009198929857E098E2B7D0022F017019F41D
:1009A0009198929803C0919A929A439526955A9558
:1009B00091F798E2A9D0417019F4919A929A02C0E5
:1009C0009198929898E2A0D0919A929A89988A9850
:1009D0002F915F914F910F910895442455249CB11C
:1009E00094E692D0A3DBA6F0953591F49FDB86F0D8
:1009F000953511F49BDB66F0492E98DB4EF0592EAD
:100A000096E082D0952D9095AADB90DBE89408952E
:100A10006894089594E178D093E0992009F0939533
:100A20009EDB84DBEEF082DBDEF06394962D97DBB9
:100A30007DDBB6F07BDBA6F0962F91DB77DB86F0D3
:100A400075DB76F0992031F0992D89DB6FDB46F06C
:100A50006DDB36F093E083DB69DB16F0E8940895F4
:100A600068940895E0E6F0E061DB3EF1903828F507
:100A70009193792E91E048D0972D909570DB56DBBD
:100A800055DBDEF0692E91937A947A94909567DB2A
:100A90004DDB772041F07A9449DB7EF0919390957D
:100AA0005EDB44DBF6CF42DB41F0933031F47090F3
:100AB000600060916200E8940895689408955F93DF
:100AC00051E17F93771BEE1CDD1C5A9521F4972F83
:100AD0007F915F910895771F791B18F4790F88949F
:100AE000F2CF0894F0CF5F93992751E1EE1CDD1C03
:100AF0005A9511F45F910895991F9A5018F4965FD2
:100B00008894F4CF0894F2CFF894222412BE7894FB
:100B10002916F1F708950F930FB6239400B30695A5
:100B20000695069500950F70BB2029F4002339F037
:100B3000A02EB02E04C00B21002309F4BB2412BE4A
:100B40000FBE0F9118950F935F930D2DDD2458E084
:100B5000E69408F4D00ED794E7945A95D1F75F91B4
:100B60000F910895FF93EF935F93E0E1F7E2EE16A4
:100B7000DF0610F055E016C0E8EEF3E0EE16DF06F3
:100B800010F054E00FC0E4E6F0E0EE16DF0610F0DF
:100B900053E008C0EAE0F0E0EE16DF0610F052E0A5
:100BA00001C051E00F3F19F0501708F4502F9BDFA0
:100BB000905D45DA0A9529F49EE241DA513009F454
:100BC00053955A95A1F75F91EF91FF9108952130C8
:100BD00019F4F8E1E0E602C0F8E1E0E88DDA089502
:100BE000203019F4F8E1E0EE11C0213019F4F9E1F8
:100BF000E0E00CC0223019F4F9E1E0E207C0233054
:100C000019F4F9E1E0E402C0F9E1E0E675DA0895EB
:100C1000203011F43FDC0895213011F450DB0895A9
:100C2000223011F4BADB0895233011F4C9DB0895A2
:040C300077DB0895D1
:10180000202020436F6E6E65637465642020202065
:1018100020506C6561736520576169742E2E2E20EF
:1018200020202020204572726F722020202020204E
:10183000204D656D6F72792045726173656420205B
:1018400020202056572D5343414E45522020202022
:101850002020562E20312E30204C69746520202007
:101860002020202020456E67696E652020202020E2
:101870002020202020202020202020202020202068
:1018800020205472616E736D697373696F6E2020CE
:101890002020202020202020202020202020202048
:1018A000202020436F6E6E656374696E6720202070
:1018B0002020202020205472792031202020202038
:1018C000202020204E6F207265706C79202020200F
:1018D0002020202020202020202020202020202008
:1018E00020312F352020204D6F64756C652020201D
:1018F0002020202020202020496E666F20202020DC
:1019000020322F352020204661756C742020202045
:1019100020202020202020436F6465732020202079
:1019200020332F35202020436C6561722020202039
:1019300020202020202020436F6465732020202059
:1019400020342F3520204D6561737572696E6720D4
:1019500020202020202020426C6F636B73202020E9
:1019600020352F35202020436C6F736520202020E8
:10197000202020202020204D6F64756C65202020C1
:00000001FF
